:020000000528D1
:080008000900031383168701B0
:100010000F309F048901880181178B1317308600E8
:1000200083128901B801983087000430A300123090
:10003000A700F422D7283808043A031DB22926085D
:1000400082070529A92905290529A929052905299D
:100050008207483441344C344934543420345434C5
:100060004F344B344D3441344B34003402080800D3
:1000700082075234453443344534503420344F34AD
:10008000433441344C3400340208080082074F34B2
:1000900054344F344D344134543449344B34203487
:1000A0004C3441345A344534523400340208080088
:1000B00082074B344F344E34543452344F344C3422
:1000C000003402080800820758342034493443348D
:1000D00049344E34203434342C34363420345434BF
:1000E000553453344C344134523449342034203460
:1000F00000340208080082075A342034493443345B
:1001000049344E34203432342C343834203454348E
:10011000553453344C344134523449340034020899
:100120000800820758343A342A342C3420345A34A4
:100130003A3423342C3420344F3452344A34493442
:100140004E343A3448342F34523400340208080014
:1001500082074934533449344E343D3420345834C2
:100160002C345A3428342B3430343034DF342C34AB
:100170002B3430343034DF342934003402080800A2
:1001800082072034203420344834413454344134FC
:100190004C344934203454345534533420342134CD
:1001A0002134213420342034003402080800AB22EA
:1001B0008207F7282A2946295A2976299B29C32903
:1001C000E829F6290A2A182A272A362A622A6D2AB5
:1001D0006E2A9E2A3808043A031D0F292608820732
:1001E0000729052905290729052905290729380887
:1001F000033A031DEA28B80A0030A6003030DB229B
:10020000A20AFA30A1009F22D7288523D7280130DF
:10021000B800A4013030DB220C30D422732C380813
:10022000063A031D1D290730B800AA013030DB2231
:10023000A20AFA30A1009F22D7283808073A031DE6
:1002400005290130B8000030A8003030DB220C3026
:10025000D4220E2C3808033A031D38290130A60099
:10026000B80A3130DB22A20AFA30A1009F22D72837
:100270003808063A031D05290130AA00B80A3130B2
:10028000DB22A20AFA30A1009F22D7283808003AC0
:10029000031D4C29FA23D7283808063A031D0529DF
:1002A0000230AA00B80A3230DB22A20AFA30A100DA
:1002B0009F22D7283808033A031D68290330A60077
:1002C000B80A3330DB22A20AFA30A1009F22D728D5
:1002D0003808063A031D05290330AA00B80A33304E
:1002E000DB22A20AFA30A1009F22D7283808033A5D
:1002F000031D84290430A600B80A3430DB22A20A88
:10030000FA30A1009F22D7283808063A031D922907
:100310000430AA00B80A3430DB22A20AFA30A10065
:100320009F22D7283808003A031D0529D623963086
:10033000A1009F22D7283808063A031D1B28053044
:10034000AA00B80A3530DB22A20AFA30A1009F22A7
:10035000D7280530A4000130B8003530DB220C303E
:10036000D422732C3808073A031D05292A08093AB4
:10037000031905290530A8000130B8003530DB220B
:100380000C30D4220E2C3808033A031DD129063034
:10039000A600B80A3630DB22A20AFA30A1009F225A
:1003A000D7283808063A031DDF290630AA00B80A04
:1003B0003630DB22A20AFA30A1009F22D728380863
:1003C000003A031D0529E8239630A1009F22D72873
:1003D0003808063A031D05290730AA00B80A373045
:1003E000DB22A20AFA30A1009F22D7283808063A59
:1003F000031D042A0830AA00B80A3830DB22A20AFA
:10040000FA30A1009F22D7283808003A031D052999
:100410000424D7283808063A031D05290930AA0004
:10042000B80A3930DB22A20AFA30A1009F22D7286D
:100430003808013A031D05290230B800CA30A2006D
:10044000D4220F30D422FA30A1009F22D7283808B6
:10045000013A031D05290530B800CF30A200D4228F
:100460000F30D422FA30A1009F22D7283808023A50
:10047000031D4C2AAC092C1C432A2D30DB22CA3028
:10048000A200D422482A2B30DB22CA30A200D42278
:10049000FA30A1009F22D7283808053A031D052904
:1004A000AE092E1C592A2D30DB22CF30A200D422D7
:1004B0005E2A2B30DB22CF30A200D422FA30A100FA
:1004C0009F22D7283808013A031D05290030B800BB
:1004D0005523FA30A1009F22D72805293808003A71
:1004E000031D822AAC01AE01AA01A801A401A60144
:1004F0001230A7000430A300B80A6D23FA30A1001F
:100500009F22D7283808023A031D902AB80ACB3018
:10051000A200D4220F30D422FA30A1009F22D72883
:100520003808053A031D0529B80AD030A200D422A4
:100530000F30D422FA30A1009F22D728D728FA30D2
:10054000A00000000000000000000000A00BA12A95
:10055000A10B9F2A08007F308600061E0134061D6D
:100560000234861C0334061C0C34BF308600061E81
:100570000434061D0534861C0634061C0D34DF3099
:100580008600061E0734061D0834861C0934061C26
:100590000E34F7308600061E0A34061D0034861C11
:1005A0000B34061C0F34103409108910880009150B
:1005B000E32209110800880009110914891009159E
:1005C000E32209110800091109108914FF3083166C
:1005D0008800831209158808881BEB2A091100304E
:1005E00083168800831208001430A1009F22091589
:1005F0003030880009111430A1009F2209153030D5
:10060000880009110530A1009F22091530308800AB
:1006100009110530A1009F223830D4220C30D42299
:100620000130D4220630D4228430D422AF012F08E6
:10063000282000380319222BDB223230A1009F2210
:10064000AF0A172BAF010630D422C530D4222F08B1
:10065000382000380319322BDB223230A1009F22D0
:10066000AF0A272BFA30A1009F220130D422AF011C
:100670008330D4222F08462000380319422BDB2276
:10068000AF0A3A2BAF01C630D4222F0858200038C9
:1006900003194D2BDB22AF0A452BAF01FA30A10025
:1006A0009F22FA30A1009F22552B0130D422AF01A6
:1006B0008030D4222F08632000380319622BDB22FC
:1006C000AF0A5A2BAF01C030D4222F087B2000384C
:1006D00003190800DB22AF0A652B0130D422AF01D9
:1006E0008030D4222F089120003803197A2BDB2286
:1006F000AF0A722BAF01C030D4222F08A8200038D7
:1007000003190800DB22AF0A7D2BAF018030D42211
:100710002F08C02000380319902BDB22AF0A882B4A
:100720000C30D422FA30A1009F223808003A031D71
:10073000A42BAF018030D4222F0863200038031986
:100740000800DB22AF0A9C2BAF018030D4222F0897
:10075000912000380319AF2BDB22AF0AA72B220808
:10076000D4220800871DB72B871107140800071D26
:10077000BC2B071187150800871CC12B8710071594
:100780000800071087140800871DC92B871107155B
:100790000800071DCE2B071187140800871CD32BD8
:1007A000871007140800071087150800871FE02B23
:1007B000071EDD2B8713071708008712071608008E
:1007C000871EE52B071387170800071287160800F6
:1007D000871FF22B071EEF2B0712871608008713BF
:1007E00007170800871EF72B871207160800071344
:1007F000871708001730B000B00BFF2B0800C42388
:100800001930A1009F22FC2B1730B000B00B092C2F
:100810000800B2231930A1009F22062C2E1C2A2C7E
:100820002A0828040319272C2A0800380319242C25
:100830001230A9000230A902AA0B1A2C280800388D
:100840000319442CA903442C1130A900442C123064
:10085000A900442C2A0828040319412C2A0800382E
:1008600003193E2C1230A9000230A907AA0B342C20
:10087000280800380319442CA90A442C1330A90075
:10088000442C1230A900442C2708123C0318492C90
:10089000502C0319552C2708123CAD0056245E2C11
:1008A00012302702AD005A245E2C5E2CFA23AD0BC9
:1008B000562C08000424AD0B5A2C08002908123CC1
:1008C0000318632C6A2C03196F2C2908123CAD0005
:1008D0005A24702C12302902AD005624702C702C32
:1008E0002908A700D7282C1C942C2608063A031D9B
:1008F0007C2C0030A500B32C2608043A031D832C61
:100900000130A500B32C2608033A031D8A2C0230BF
:10091000A500B32C2608013A031D912C0330A50035
:10092000B32C0430A500B32C2608063A031D9B2CDB
:100930000830A500B32C2608043A031DA22C07306A
:10094000A500B32C2608033A031DA92C0630A500E8
:10095000B32C2608013A031DB02C0530A500B32C9A
:100960000430A500B32C2308043C0318B82CBF2C7A
:100970000319C42C2308043CAB00C524D32C043039
:100980002302AB00CC24D32CD32CE8239630A10037
:100990009F22AB0BC52C0800D6239630A1009F22C6
:1009A000AB0BCC2C08002508043C0318D82CDF2CFA
:1009B0000319E42C2508043CAB00CC24E52C0430BE
:1009C0002502AB00C524E52CE52C2508A300D7287B
:02400E00F13F80
:00000001FF
